:0200000068286E
:100008008C00030E83018E000A088D0033281030FF
:10001800C3008F01AB01C40CC50C031C192841088F
:10002800AB0703188F0A40088F070310C10DC00DD6
:10003800C30B0F282B080800260803193228A5012E
:10004800FF3025029201031C920A120803192F2877
:10005800A50A25032428A603260A202808000B1130
:1000680020089F0A0319A00A1108900A0319910A87
:100078006A301002AE001108AF00031CAF0318303D
:10008800AF02AD01AF1FAD0A2D0803194D2890012D
:10009800910135301F02AE002008AF00031CAF03EA
:1000A8000C30AF02B001AF1FB00A30080319602846
:1000B8009F01A0010130C20083010D088A000E0EC5
:1000C80083008C0E0C0E090083169F01A00190017D
:1000D80091019601970101308100FF30850086016A
:1000E8008312860181018B1603118B179A01073041
:1000F8001A0292009301921B930A130803198C2881
:100108001A08313E8313840080019A0A1A037B2857
:100118009A0106301A0294009501941B950A150855
:100128000319E52B1A08313E831384000008C50023
:10013800C4011030C100C0010B20A2000F08A300A9
:100148001A08A2070318A30A00019A1BFF30A30785
:10015800220899001A089C0000301C020319C928BB
:1001680001301C020319132902301C0203195D29EE
:1001780003301C020319EF2904301C020319802ADA
:1001880005301C020319C92A112B82301002A8005D
:100198001108A900031CA9031430A9029801A91B7E
:1001A800980A18089D000319E72810081D3CA800A4
:1001B8001030A900031CA9031108A9029801A91B62
:1001C800980A18089D001D089400031D0B290B3080
:1001D8001002A8001108A900031CA9031330A902E2
:1001E8009801A91B980A18089D00031909291008E5
:1001F800A63CA8000E30A900031CA9031108A902F7
:100208009801A91B980A18089D001D089400140855
:1002180003191229083019079D009900112BA030E5
:100228001002A8001108A900031CA9030F30A90295
:100238009B01A91B9B0A1B08980003193129100868
:10024800B23CA8000C30A900031CA9031108A9029C
:100258009B01A91B9B0A1B08980018089D00031DF9
:10026800552976301002A8001108A900031CA9031B
:100278001630A9029B01A91B9B0A1B0898000319A9
:1002880053291008883CA8001330A900031CA903AF
:100298001108A9029B01A91B9B0A1B0898001808B2
:1002A8009D001D0803195C2908301907980099005A
:1002B800112BAC301002A8001108A900031CA903D7
:1002C8000D30A9028F01A91B8F0A0F089E00031980
:1002D8007B291008B23CA8000C30A900031CA90314
:1002E8001108A9028F01A91B8F0A0F089E001E087A
:1002F800A100031D9F2970301002A8001108A90051
:10030800031CA9031730A9028F01A91B8F0A0F0824
:100318009E0003199D291008F33CA8001630A90077
:10032800031CA9031108A9028F01A91B8F0A0F0832
:100338009E001E08A10021089B00031DC32935301B
:100348001002A8001108A900031CA9030C30A90277
:100358009E01A91B9E0A1E08A1000319C1291008A5
:10036800BE3CA8000A30A900031CA9031108A90271
:100378009E01A91B9E0A1E08A10021089B001B08BC
:100388009800031DE72976301002A8001108A9007B
:10039800031CA9031630A902A101A91BA10A21085F
:1003A8009B000319E52910087C3CA8001530A9001A
:1003B800031CA9031108A902A101A91BA10A21086C
:1003C8009B001B08980018080319EE290830190724
:1003D8009B009900112B77301002A8001108A90082
:1003E800031CA9030130A902A401A91BA40A24081B
:1003F8008F0003190C2A1008003CA800A901031C4F
:10040800A9031108A902A401A91BA40A24088F00A2
:100418000F089E00031D302A35301002A80011086D
:10042800A900031CA9030C30A902A401A91BA40A52
:1004380024088F0003192E2A1008BE3CA8000A3091
:10044800A900031CA9031108A902A401A91BA40A55
:1004580024088F000F089E001E08A100031D542ABF
:1004680041301002A8001108A900031CA9030A3092
:10047800A9028F01A91B8F0A0F089E000319522A8F
:100488001008473CA8000930A900031CA90311085B
:10049800A9028F01A91B8F0A0F089E001E08A10040
:1004A80021089B00031D782A6A301002A800110851
:1004B800A900031CA9031830A9029E01A91B9E0AC2
:1004C8001E08A1000319762A1008F33CA80016306C
:1004D800A900031CA9031108A9029E01A91B9E0AD1
:1004E8001E08A10021089B001B0803197F2A083059
:1004F8001907A1009900112B6B301002A8001108F0
:10050800A900031CA9030330A9028F01A91B8F0AA4
:100518000F089E0003199D2A10087D3CA800A90118
:10052800031CA9031108A9028F01A91B8F0A0F0830
:100538009E001E08A100031DC12A41301002A80018
:100548001108A900031CA9030A30A9028F01A91BDD
:100558008F0A0F089E000319BF2A1008533CA800F1
:100568000730A900031CA9031108A9028F01A91BC0
:100578008F0A0F089E001E08A10021080319C82A27
:10058800083019079E009900112B4D301002A80061
:100598001108A900031CA9030830A902A401A91B7A
:1005A800A40A24088F000319E72A1008E83CA800C9
:1005B8000330A900031CA9031108A902A401A91B5F
:1005C800A40A24088F000F089E00031D0B2BD630A9
:1005D8001002A8001108A900031CA9030630A902EB
:1005E800A401A91BA40A24088F000319092B1008C9
:1005F800713CA8000230A900031CA9031108A90234
:10060800A401A91BA40A24088F000F089E001E0835
:100618000319112B0830190799008312190886004D
:100628000430A60020208312FF308600A40142086F
:10063800031DA40A240803196F2BC201B10A31084B
:10064800093CBF01031CBF0A3F0803192E2BB10147
:10065800B20A32033208053CBE01031CBE0A3E083A
:100668000319392BB201B30A33033308093CBD011E
:10067800031CBD0A3D080319442BB301B40A340313
:100688003408053CBC01031CBC0A3C0803194F2B69
:10069800B401B50A35033508093CBB01031CBB0A84
:1006A8003B0803195A2BB501B60A36033608013C34
:1006B8008F01031C8F0A0F08BA0003196A2B35082B
:1006C800033C8F01031C8F0A0F08BA003A0803196C
:1006D8006F2BB501B6018312050899009C00033001
:1006E8001C020319802B05301C020319832B0630CA
:1006F8001C020319AD2BE22BB101B201E22B170842
:10070800960A0319970A1608643CA800A901031C55
:10071800A9031708A902A701A91BA70A27080319F3
:10072800AC2B96019701B30A3308093CB901031CA5
:10073800B90A39080319A32BB301B40A34033408DE
:10074800053CB801031CB80A38080319AC2BB401DE
:10075800E22B1708960A0319970A1608643CA800A2
:10076800A901031CA9031708A902AA01A91BAA0A1F
:100778002A080319E22B96019701B50A3508093CA6
:10078800B701031CB70A37080319CD2BB501B60A00
:1007980036033608013C8F01031C8F0A0F08AC0092
:1007A8000319DD2B3508033C8F01031C8F0A0F0842
:1007B800AC002C080319E22BB501B6019A0A1A03FA
:0607C8008D288C28E62BB1
:02400E00FA3F77
:00000001FF
